:020000040000FA
:0600000001EF1DF01200EB
:020006001200E6
:0600080024EF09F01200D4
:02000E000100EF
:0C001000343A000000010000FC00000079
:04001C00D9CFE6FF53
:10002000E1CFD9FFFE0EDB50006E016A013404E21D
:1000300000500008000E015403E2FE0EDB06F2D76A
:10004000E552E7CFD9FF1200D9CFE6FFE1CFD9FFC4
:10005000FE0EDB50E66EADEC1CF0E552E552E7CF4C
:10006000D9FF1200D9CFE6FFE1CFD9FF030EE12679
:10007000FE0EDB50006E016A013404E200505F089E
:10008000000E015401E2A3D0FD0EDB50006E016AA8
:10009000013404E200503F08000E015401E297D001
:1000A000FD0EDB50026E036A080E256E266A02C042
:1000B00020F003C021F0B6EC16F020C002F021C001
:1000C00003F0600E0302F3CF03F00202F3CF02F05D
:1000D000F4500326FE0EDB5000010224006E000ED9
:1000E0000320016E00C0DEFF01C0DDFFFD0EDB500E
:1000F000026E036AFD0EDB50046E056A080E256E63
:10010000266A04C020F005C021F0B6EC16F020C02D
:1001100004F021C005F0030ED89004360536E80639
:10012000FBE10450025C006E05500358016E020EA4
:1001300000C0DBFFFC0EDB50006E016A00500110B6
:1001400014E1020EDB500FEC1DF0F3CF00F0F4CF02
:1001500001F0001E011EDECFE9FFDDCFEAFF5F0EDA
:10016000E926020EEA220050EF16FC0EDB50006E6C
:10017000016A010E001801E1015010E1020EDB508E
:100180000FEC1DF0F3CF00F0DECFE9FFDDCFEAFF8B
:100190005F0EE926020EEA220050EF12FC0EDB5041
:1001A000006E016A020E001801E1015010E1020E1A
:1001B000DB500FEC1DF0F3CF00F0DECFE9FFDDCF19
:1001C000EAFF5F0EE926020EEA220050EF1A030E44
:1001D000E15C02E2E16AE552E16EE552E7CFD9FF68
:1001E0001200D9CFE6FFE1CFD9FF0A0EE126FB0EC0
:1001F000DB50026E036AFD0EDB50046E056A04508C
:10020000025C006E05500358016E020E00C0DBFF59
:10021000030E01C0DBFFFC0EDB50026E036AFE0E14
:10022000DB50046E056A0450025C006E05500358F2
:10023000016E00C0DEFF01C0DDFF020EDBCF00F06B
:10024000030EDBCF01F00001800E011415E02068E1
:100250002168020EDBCF25F0030EDBCF26F0DCECAD
:1002600016F0020E1EC0DBFF030E1FC0DBFF060EE2
:10027000DB68070EDB6807D0010EF36E060EF3CFC6
:10028000DBFF070EDB6ADECF00F0DDCF01F00001FF
:10029000800E011411E020682168DECF25F0DDCF4B
:1002A00026F0DCEC16F01EC0DEFF1FC0DDFF040EE2
:1002B000DB68050EDB6807D0010EF36E040EF3CF8A
:1002C000DBFF050EDB6AD9CFE9FFDACFEAFF010ECB
:1002D000D890EE36ED36E806FBE1D950020FE96E14
:1002E000DACFEAFF010ED890EE36ED36E806FBE1F4
:1002F000FA0EDB50E66EFD0EDB50E66EFE0EDB50B6
:10030000E66EB0DEE552E552E552DECF00F0DDCF1D
:1003100001F0020EDBCF02F0030EDBCF03F003503F
:100320000118E8AE02D0013404D00050025C015044
:1003300003586EE2DECF02F0DDCF03F0D890033237
:100340000232020EDBCF20F0030EDBCF21F0025091
:10035000205C006E03502158016E080E00C0DBFFC8
:10036000090E01C0DBFFFE0EDB50006E016AFC0EC1
:10037000DB50026E036A0250001802E103500118BC
:1003800046E0080EDBCF00F0090EDBCF01F00001E4
:10039000800E011416E1FD0EDBCFE7FF060EDB50E9
:1003A000E726FD0EE7CFDBFFDECF00F0DDCF01F06B
:1003B000D950080FE96EDACFEAFF0050EE5E015027
:1003C000ED5AFE0EDBCFE7FF040EDB50E726FE0EF4
:1003D000E7CFDBFF020EDBCF00F0030EDBCF01F037
:1003E000D950080FE96EDACFEAFF0050EE2601502F
:1003F000ED22FA0EDB50E66EFD0EDB50E66EFE0ED1
:10040000DB50E66E2FDEE552E552E552ACD769D0FF
:10041000020EDBCF02F0030EDBCF03F0D8900332E5
:1004200002320250DE5C006E0350DD58016E080E91
:1004300000C0DBFF090E01C0DBFFFD0EDB50006ECC
:10044000016AFB0EDB50026E036A0250001802E1E3
:100450000350011846E0080EDBCF00F0090EDBCF99
:1004600001F00001800E011418E1FE0EDBCFE7FF62
:10047000040EDB50E726FE0EE7CFDBFF020EDBCFDC
:1004800000F0030EDBCF01F0D950080FE96EDACF90
:10049000EAFF0050EE5E0150ED5AFD0EDBCFE7FFA4
:1004A000060EDB50E726FD0EE7CFDBFFDECF00F0C8
:1004B000DDCF01F0D950080FE96EDACFEAFF005026
:1004C000EE260150ED22FA0EDB50E66EFD0EDB50FB
:1004D000E66EFE0EDB50E66EC5DDE552E552E552F6
:1004E000ACD70A0EE15C02E2E16AE552E16EE55248
:1004F000E7CFD9FF1200D9CFE6FFE1CFD9FF020E37
:10050000E126E66AE66A0FDBE552E5520101D06BAF
:10051000D16BDE6ADD6ADECF00F0DDCF01F0000EC8
:10052000005C030E015811E2DECFE9FFDDCFEAFFE8
:100530005F0EE926020EEA22EF50E66EA2DAE552DD
:10054000DF2A010E01E3DB2AE6D7020EE15C02E2BC
:10055000E16AE552E16EE552E7CFD9FF1200D9CF4B
:10056000E6FFE1CFD9FFFA0EDB50E66EFD0EDB5061
:10057000E66EFC0EDB50E66EFD0EDB50E66EFE0E08
:10058000DB50E66E2EDE006E050EE15E0050FA0EC8
:10059000DB50E66EFB0EDB50E66EFC0EDB50E66ECB
:1005A000FD0EDB50E66EFC0EDB50E66E1ADE006ED2
:1005B000050EE15E0050FA0EDB50E66EFB0EDB50DE
:1005C000E66EFE0EDB50E66EFB0EDB50E66EFC0EBA
:1005D000DB50E66E06DE006E050EE15E0050FA0EA0
:1005E000DB50E66EFD0EDB50E66EFE0EDB50E66E77
:1005F000FB0EDB50E66EFE0EDB50E66EF2DD006EAB
:10060000050EE15E005077DFE552E7CFD9FF12001B
:10061000D9CFE6FFE1CFD9FF050EE126030EDB6A55
:10062000FD0EDB50026E036AFE0EDB50046E056A9F
:100630000450025C006E05500358016E040E00C0A9
:10064000DBFFFC0EDB50E76E020EE7CFDBFFFC0E9C
:10065000DB50026E036A020E206E216A02C025F092
:1006600003C026F0DCEC16F01EC000F01FC001F045
:10067000030ED8800056000E015600C0DEFF01C0F8
:10068000DDFF030EDB50006E016A020EDB50026ECE
:10069000036A03500118E8AE02D0013404D00050C0
:1006A000025C0150035801E276D1FB0EDB50E66E8E
:1006B000FD0EDBCF00F0020EDB500024E66EFE0ED6
:1006C000DBCF01F0030EDB500124E66ECBDCE552FC
:1006D000E552E552FB0EDB50E66EFD0EDB50026E7E
:1006E000036A020EDB50046E056A0450025C006E61
:1006F00005500358016E0050E66EFE0EDBCF06F08B
:10070000030EDB500624E66EADDCE552E552E55201
:10071000FB0EDB50E66EFD0EDBCF00F0020EDB5071
:100720000024E66EFE0EDB50036E046A030EDB50FF
:10073000056E066A0550035C016E06500458026E91
:100740000150E66E8FDCE552E552E552FB0EDB50C0
:10075000E66EFD0EDB50026E036A020EDB50046E85
:10076000056A0450025C006E05500358016E00508B
:10077000E66EFE0EDB50086E096A030EDB500A6E51
:100780000B6A0A50085C066E0B500958076E06503B
:10079000E66E68DCE552E552E552FB0EDB50E66E94
:1007A000FD0EDBCF00F0030EDB500024E66EFD0EE5
:1007B000DBCF05F0020EDB500524036E046A000E49
:1007C0000422040EDB50066E076A0650035C016EBD
:1007D00007500458026E0150E66E44DCE552E552C3
:1007E000E552FB0EDB50E66EFD0EDB50026E036A37
:1007F000030EDB50046E056A0450025C006E055067
:100800000358016E0050E66EFD0EDBCF0AF0020EBB
:10081000DB500A24086E096A000E0922040EDB5020
:100820000B6E0C6A0B50085C066E0C500958076E74
:100830000650E66E17DCE552E552E552FB0EDB5042
:10084000E66EFD0EDBCF00F0030EDB500024E66EFB
:10085000FD0EDB50056E066A020EDB50076E086A5D
:100860000750055C036E08500658046E040EDB50FA
:10087000096E0A6A0950035C016E0A500458026E40
:100880000150E66E32EC00F0E552E552E552FB0E07
:10089000DB50E66EFD0EDB50026E036A030EDB508A
:1008A000046E056A0450025C006E05500358016E28
:1008B0000050E66EFD0EDB500A6E0B6A020EDB5036
:1008C0000C6E0D6A0C500A5C086E0D500B58096EC8
:1008D000040EDB500E6E0F6A0E50085C066E0F5051
:1008E0000958076E0650E66E32EC00F0E552E5520C
:1008F000E552DECF00F0DDCF01F00001800E0114E3
:100900001EE0030EDB50026E036A040E206E216AA5
:1009100002C025F003C026F0DCEC16F01EC000F08B
:100920001FC001F0060E0026000E0122D9CFE9FFFC
:10093000DACFEAFF0050EE260150ED2229D0030E57
:10094000DB50046E056A020EDB50066E076A065025
:10095000045C026E07500558036E040E206E216A77
:1009600002C025F003C026F0DCEC16F01EC000F03B
:100970001FC001F00A0E0026000E0122D9CFE9FFA8
:10098000DACFEAFF0050EE260150ED22020EDB0620
:10099000030EDB2A76D6AFDD050EE15C02E2E16AEA
:1009A000E552E16EE552E7CFD9FF120082828290D4
:1009B0008294960EE66E24EC00F0E55282808284EA
:1009C000640EE66E24EC00F0E552210EE66E3FD890
:1009D000E552900EE66E3BD8E552050EE66E37D82E
:1009E000E552130EE66E33D8E552200EE66E2FD890
:1009F000E552960EE66E24EC00F0E5520C0EE66E23
:100A000026D8E552320EE66E24EC00F0E5521200D4
:100A10008290E66AE66A87D8E552E5520201446BA5
:100A2000456BD890455104E6000E445D030E4559D0
:100A30000DE2E66A26D8E5520A0EE66E0EEC00F0EC
:100A4000E5520201442B000E4523EBD71200D9CF0B
:100A5000E6FFE1CFD9FF82928290190EE66E0EEC8E
:100A600000F0E552FE0EDBCF00F0016A00BE016827
:100A70000050E66E20D8E5528280E552E7CFD9FFDC
:100A80001200D9CFE6FFE1CFD9FF82828290190E02
:100A9000E66E0EEC00F0E552FE0EDBCF00F0016AD0
:100AA00000BE01680050E66E06D8E5528280E5522D
:100AB000E7CFD9FF1200D9CFE6FFE1CFD9FFE65249
:100AC000080EDF6EDFCF00F0016A00BE016801345E
:100AD00004E200500008000E015420E282960A0E43
:100AE000E66E0EEC00F0E552FE0EDBCF00F0016A80
:100AF00000BE01680050800B02E1829801D082881C
:100B00008286FE0EDBCF00F0016A00BE0168D8903D
:100B10000036013600C0DBFFDF06D4D7E552E552D0
:100B2000E7CFD9FF1200D9CFE6FFE1CFD9FFFD0E05
:100B3000DB50006E016A070E0016000E0116400E13
:100B40000010E66E84DFE552FE0EDB50006E016A97
:100B50007F0E0016000E0116800E0010E66E77DF85
:100B6000E552E552E7CFD9FF1200D9CFE6FFE1CF3A
:100B7000D9FFE652DF6ADFCF00F0016A00BE0168EC
:100B8000D890015004E65B0E005C000E01581CE298
:100B9000FE0EDB50E66EDFCF00F0016A00BE01689A
:100BA0000050E66EC0DFE552E552E66A200EE66EC2
:100BB000A3D8E552E552DFCF00F0016A00BE01681C
:100BC000060E0024DF6ED7D7FE0EDB50E66EE66A17
:100BD000AADFE552E552E552E552E7CFD9FF120010
:100BE000D9CFE6FFE1CFD9FF020EE126E66AE66A39
:100BF0009ADFE552E552DE6ADD6ADECF00F0DDCF36
:100C000001F0D890015004E6600E005C000E01581F
:100C100025E2E66A36DFE552E66A33DFE552E66A48
:100C200030DFE552E66A2DDFE552E66A2ADFE5525B
:100C3000E66A27DFE552E66A24DFE552E66A21DF4D
:100C4000E552DECF00F0DDCF01F0080E0026000EE9
:100C5000012200C0DEFF01C0DDFFCFD7E66AE66AF1
:100C600062DFE552E552020EE15C02E2E16AE55222
:100C7000E16EE552E7CFD9FF1200D9CFE6FFE1CF11
:100C8000D9FFE652DF6ADFCF00F0016A00BE0168DB
:100C9000D890015004E6080E005C000E015827E2CF
:100CA000DFCF00F0016A00BE01680050E66EFE0E64
:100CB000DB50E66E38DFE552E552E66AE2DEE552E9
:100CC000E66ADFDEE552E66ADCDEE552E66AD9DE98
:100CD000E552E66AD6DEE552E66AD3DEE552E66A1A
:100CE000D0DEE552E66ACDDEE552DF2ACCD7E5520A
:100CF000E552E7CFD9FF1200D9CFE6FFE1CFD9FF08
:100D0000FE0EDB500201466F4651006E016AD8901C
:100D1000015004E6200E005C000E015801E287D06D
:100D20004651006E016A013404E200507F08000E53
:100D3000015401E27CD0476B4751006E016AD890A4
:100D4000015004E6050E005C000E01586DE24651AC
:100D5000006E016AD890015004E6500E005C000E4F
:100D6000015825E24651006E016A200E005E000E19
:100D7000015A050E0102F3CF01F00002F3CF00F09B
:100D8000F450012600C048F247514825F66EF76A34
:100D9000000EF722B80EF626300EF7220800F5CF27
:100DA00000F0016A00BE016800C049F224D046513B
:100DB000006E016A500E005E000E015A050E01021F
:100DC000F3CF01F00002F3CF00F0F450012600C091
:100DD00048F247514825F66EF76A000EF722A80E32
:100DE000F626310EF7220800F5CF00F0016A00BEAA
:100DF000016800C049F24951E66E43DEE552FD0E3E
:100E0000DBCF00F0016A00BE0168013404E200504B
:100E10000008000E015405E202014951E66E31DE80
:100E2000E5520201472B88D7E66A2BDEE552E552F0
:100E3000E7CFD9FF1200D9CFE6FFE1CFD9FFE652C5
:100E400002014B6B4C6B4D6B4E6BDF6ADFCF00F0DA
:100E5000016A00BE0168FD0EDB50026E036A02509B
:100E6000001802E10350011807E0D8904B374C37C7
:100E70004D374E37DF2AEAD74B834BC24FF24CC275
:100E800050F24DC251F24EC252F2506B516B526B46
:100E9000080E1F0B4BC253F24CC254F24DC255F216
:100EA0004EC256F208E00201D890563355335433FF
:100EB0005333E806F9E10201546B556B566B100E83
:100EC0001F0B4BC257F24CC258F24DC259F24EC2E0
:100ED0005AF208E00201D8905A3359335833573345
:100EE000E806F9E10201586B596B5A6B180E1F0B9B
:100EF0004BC25BF24CC25CF24DC25DF24EC25EF27E
:100F000008E00201D8905E335D335C335B33E80662
:100F1000F9E102015C6B5D6B5E6B010EE66EFE0E2D
:100F2000DB50E66E00DEE552E5525BC2E6FF2AD8F2
:100F3000E552020EE66EFE0EDB50E66EF4DDE55283
:100F4000E55257C2E6FF1ED8E552030EE66EFE0ECE
:100F5000DB50E66EE8DDE552E55253C2E6FF12D8FB
:100F6000E552040EE66EFE0EDB50E66EDCDDE55269
:100F7000E5524FC2E6FF06D8E552E552E552E7CF0B
:100F8000D9FF1200D9CFE6FFE1CFD9FFE652828226
:100F90008290080EDF6EDFCF00F0016A00BE0168AC
:100FA000013404E200500008000E015420E2829651
:100FB0000A0EE66E0EEC00F0E552FE0EDBCF00F0FE
:100FC000016A00BE01680050010B02E1829801D065
:100FD00082888286FE0EDBCF00F0016A00BE0168C7
:100FE000D8900132003200C0DBFFDF06D4D7828008
:100FF000E552E552E7CFD9FF1200E66AB6DDE552C9
:10100000010EE66EB2DDE552020EE66EAEDDE55291
:10101000030EE66EAADDE552040EE66EA6DDE5528D
:10102000050EE66EA2DDE552060EE66E9EDDE55289
:10103000070EE66E9ADDE5521200D9CFE6FFE1CF4A
:10104000D9FFFD0EDB50E66EFE0EDB50E66E6BDD6B
:10105000E552E552E66A200EE66E4EDEE552E552B6
:10106000E552E7CFD9FF1200E66A0BDDE552040E28
:10107000E66E07DDE552020EE66E03DDE5527F0EF9
:10108000E66EFFDCE552020EE66EFBDCE552040E76
:10109000E66EF7DCE552E66AF4DCE552E66AF1DC7E
:1010A000E5521200100EE66EECDCE552200EE66E04
:1010B000E8DCE5527F0EE66EE4DCE552200EE66EDB
:1010C000E0DCE552100EE66EDCDCE552E66AD9DCC7
:1010D000E552E66AD6DCE552E66AD3DCE552120058
:1010E000080EE66ECEDCE5521C0EE66ECADCE5525A
:1010F0002A0EE66EC6DCE552080EE66EC2DCE5524C
:10110000080EE66EBEDCE552F80EE66EBADCE5527D
:10111000E66AB7DCE552E66AB4DCE5521200080E76
:10112000E66EAFDCE552080EE66EABDCE5522A0E49
:10113000E66EA7DCE5521C0EE66EA3DCE552080E57
:10114000E66E9FDCE552E66A9CDCE552E66A99DCD5
:10115000E552E66A96DCE5521200E66A92DCE55258
:10116000060EE66E8EDCE552090EE66E8ADCE5526E
:10117000090EE66E86DCE552060EE66E82DCE5526E
:10118000E66A7FDCE552E66A7CDCE552E66A79DCF9
:10119000E5521200E66A75DCE552060EE66E71DC79
:1011A000E5520F0EE66E6DDCE5520F0EE66E69DC61
:1011B000E552060EE66E65DCE552E66A62DCE55253
:1011C000E66A5FDCE552E66A5CDCE5521200D9CFE4
:1011D000E6FFE1CFD9FFFD0EDBCFE9FFFE0EDBCF4F
:1011E000EAFFEFCF00F0016A00BE01680050011075
:1011F00027E0FC0EDBCF00F0016A00BE0168005062
:10120000E66EFD0EDBCFE9FFDB2AFE0EDBCFEAFF49
:1012100001E3DB2AEFCF02F0036A02BE036802504B
:10122000E66E6ADDE552E552C80EE66EE66AE66AEB
:10123000E66A33EC11F0E552E552E552E552CBD7C0
:10124000E552E7CFD9FF1200DACFE4FFE2CFDAFFB1
:10125000E9CFE4FFEACFE4FFF6CFE4FFF7CFE4FF06
:10126000F5CFE4FFF3CFE4FFF4CFE4FFFACFE4FFE0
:1012700000EE18F0140EE80403E3EECFE4FFFBD712
:1012800000EE00F0180EE80403E3EECFE4FFFBD716
:10129000E652D9CFE6FFE1CFD9FFE6529E50200BB0
:1012A00001E0010E2C6E2D6A2C502D1001E195D01D
:1012B00072EC1CF0DF6EAB50040B01E0010E2E6EE1
:1012C0002F6A2E502F100BE1AB50020B01E0010EE4
:1012D000306E316A3050311002E1000E01D0010E43
:1012E0002C6E2D6A2C502D1002E0AB98AB88AC50C0
:1012F000020B01E0010E2C6E2D6A2C502D1001E125
:10130000F6D78150020B01E0010E2C6E2D6A2C5095
:101310002D100AE1DFCF2CF02D6A2CBE2D682C5049
:10132000E66EC4EC1CF0E552DFCF2CF02D6A2CBE2B
:101330002D68080E2C1801E12D500FE19FC22CF0F2
:101340002D6A2CBE2D682D3404E22C500008000EAE
:101350002D5402E202019F0740D0DFCF2EF02F6A0A
:101360002EBE2F680D0E2E1801E12F500DE09FC2EA
:1013700030F0316A30BE3168D890315004E65A0EF0
:10138000305C000E315802E3000E01D0010E2C6ECD
:101390002D6A2C502D1013E0DFCF2CF02D6A2CBEBF
:1013A0002D6802019F519F2BE96EEA6AE9BEEA6847
:1013B0006E0EE926010EEA222CC0EFFF0ED09FC26E
:1013C000E9FFEA6AE9BEEA686E0EE926010EEA2242
:1013D000EF6A02019F6B010E046F9E50010B2C6E91
:1013E0002D6A010E2C1801E12D5018E10201002B8D
:1013F000000E0123040ED8800055000E015505E2B1
:10140000006B016B010E0E6F0F6BDB0EE66E0B0EA9
:10141000E66E91EC1CF0E552E5529E90E552E552E5
:10142000E7CFD9FFE55200EE17F0180EE80403E30A
:10143000E5CFEDFFFBD700EE2BF0140EE80403E33D
:10144000E5CFEDFFFBD7E5CFFAFFE5CFF4FFE5CF22
:10145000F3FFE5CFF5FFE5CFF7FFE5CFF6FFE5CFEB
:10146000EAFFE5CFE9FFE5CFDAFF1100200EE66ED7
:10147000E66A7C0EE66EB5EC1BF0E552E552E552ED
:10148000F28CF28E100EE66E270EE66EE66AE66AC3
:1014900033EC11F0E552E552E552E5521200D9CF96
:1014A000E6FFE1CFD9FF020EE126DE6ADD6AFD0E1E
:1014B000DBCFE9FFFE0EDBCFEAFFEFCF00F0016AE2
:1014C00000BE0168005001101CE0FD0EDBCFE9FFFB
:1014D000FE0EDBCFEAFFEFCF00F0016A00BE01682D
:1014E00000C0E6FF01C0E6FF1FD8E552E552DF2A43
:1014F000010E01E3DB2AFD0EDB2AFE0E01E3DB2AEF
:10150000D6D7DECF00F0DDCF01F000C0F3FF01C081
:10151000F4FF020EE15C03E200D0E16AE552E16E05
:10152000E552E7CFD9FF1200D9CFE6FFE1CFD9FFCF
:10153000AC50020B01E0010E006E016A0050011078
:1015400001E1F6D7FD0EDBCFE6FFC4EC1CF0E5525F
:10155000E552E7CFD9FF12000D0EE66EE66AE4DF32
:10156000E552E5520A0EE66EE66ADEDFE552E55226
:101570001200D9CFE6FFE1CFD9FF0A0EE126020122
:101580005C0E026F010E036FFC0EDBCF00F0016AF0
:1015900000BE0168013404E200500108000E01544D
:1015A00001E214D1FC0EDBCF00F0016A00BE01683D
:1015B0000050011028E1FD0EDBCF00F0FE0EDBCF66
:1015C00001F0060E00C0DBFF070E01C0DBFF080EB6
:1015D000DB6A090EDB6A02C2E6FF03C2E6FFD950EE
:1015E000060FE96EDACFEAFFEECFE6FFEECFE6FFB9
:1015F000EECFE6FFEFCFE6FFA9EC1AF0006E060E85
:10160000E15E005010D002C2E6FF03C2E6FFFD0E0D
:10161000DBCFE6FFFE0EDBCFE6FF0FEC1AF0E55264
:10162000E552E552E55202010D51400B01E0010E79
:10163000006E016A0050011001E191D05C0EE66E6F
:10164000010EE66E43EC1CF0E552E552020EF3CFBC
:10165000DBFF030EF4CFDBFFDE6ADD6ADECF00F0D6
:10166000DDCF01F0020EDBCF02F0030EDBCF03F083
:101670000250005C0350015831E2020EDBCF02F051
:10168000030EDBCF03F0DE50025CE96EDD50035841
:10169000EA6EE906000EEA5A5C0EE926010EEA221D
:1016A000EF50E66EFC0EDBCF00F0016A00BE016871
:1016B000040E0026000E0122DE50005CE96EDD50B3
:1016C0000158EA6E5C0EE926010EEA22E552E75067
:1016D000EF6EDF2A010E01E3DB2AC0D7DE6ADD6A86
:1016E000DECF00F0DDCF01F0FC0EDBCF04F0056AA9
:1016F00004BE0568050E0426000E0522020EDB500E
:10170000045C026E030EDB500558036E0250005C51
:101710000350015824E202010D51100B01E0010EAB
:10172000006E016A005001100BE0DECFE9FFDDCF53
:10173000EAFF5C0EE926010EEA22300EEF6E0AD0B7
:10174000DECFE9FFDDCFEAFF5C0EE926010EEA22DB
:10175000200EEF6EDF2A010E01E3DB2AC1D7FC0E5B
:10176000DBCFE9FFEA6AE9BEEA68050EE926000E6A
:10177000EA225C0EE926010EEA22EF6A02010D510F
:10178000800B01E0010E006E016A0050011011E0B3
:10179000FB0EDBCF00F0016A00BE01680050E66E70
:1017A00002C2E6FF03C2E6FF12DDE552E552E55252
:1017B0000DD002C2E6FF03C2E6FF71DEE552E5523C
:1017C000020EF3CFDBFF030EF4CFDBFF0A0EE15C6A
:1017D00002E2E16AE552E16EE552E7CFD9FF12007D
:1017E000D9CFE6FFE1CFD9FF0E0EE126F90EDBCF10
:1017F000DEFFDBCFDDFFF80EDBCF02F0036A02BEB7
:101800000368033404E202500008000E035404E3AA
:10181000070E006E016A1BD0F80EDBCF04F0056ADC
:1018200004BE0568053404E204501608000E055491
:1018300004E2170E006E016A0AD0F80EDBCF00F04A
:10184000016A00BE0168010E0026000E0122080E8A
:1018500000C0DBFF090E01C0DBFF020EDB6A030ED6
:10186000DB6AFB0EDBCF00F0FC0EDBCF01F0FD0EE0
:10187000DBCF02F0FE0EDBCF03F0246A256A266A76
:10188000276A00C01FF001C020F002C021F003C091
:1018900022F078EC17F0010A33E1F90EDBCFE9FF13
:1018A000DB2AFA0EDBCFEAFF01E3DB2A2D0EEF6E17
:1018B000FB0EDBCF00F0FC0EDBCF01F0FD0EDBCF2B
:1018C00002F0FE0EDBCF03F0246A256A800E266E3E
:1018D000BF0E276E00C01FF001C020F002C021F033
:1018E00003C022F049EC16F0FB0E1FC0DBFFFC0E1C
:1018F00020C0DBFFFD0E21C0DBFFFE0E22C0DBFFA0
:10190000FB0EDBCF00F0FC0EDBCF01F0FD0EDBCFDA
:1019100002F0FE0EDBCF03F0246A256A266A276AEE
:1019200000C01FF001C020F002C021F003C022F06F
:101930006FEC17F0010A4AE1FB0EDBCF00F0FC0E62
:10194000DBCF01F0FD0EDBCF02F0FE0EDBCF03F0AC
:10195000246A256A800E266E3F0E276E00C01FF097
:1019600001C020F002C021F003C022F078EC17F093
:10197000010A2CE1006A016A200E026E410E036E1C
:10198000D950FB0FE96EFF0EDA20EA6EEECF1FF0A2
:10199000EECF20F0EECF21F0EFCF22F000C024F008
:1019A00001C025F002C026F003C027F049EC16F074
:1019B00022C0EDFF21C0EDFF20C0EDFF1FC0EFFFF3
:1019C000020EDB06030E01E2DB06B6D7FB0EDBCF11
:1019D00000F0FC0EDBCF01F0FD0EDBCF02F0FE0EBF
:1019E000DBCF03F0246A256A200E266E410E276E97
:1019F00000C01FF001C020F002C021F003C022F09F
:101A000078EC17F0010A2EE0FB0EDBCF00F0FC0EA5
:101A1000DBCF01F0FD0EDBCF02F0FE0EDBCF03F0DB
:101A2000246A256A200E266E410E276E00C01FF024
:101A300001C020F002C021F003C022F0F6EC15F046
:101A4000FB0E1FC0DBFFFC0E20C0DBFFFD0E21C024
:101A5000DBFFFE0E22C0DBFF020EDB2A030E01E3DA
:101A6000DB2AB4D7020EDBCF00F0030EDBCF01F090
:101A7000D950080FE96EDACFEAFF0050EE26015088
:101A8000ED22010EF36E040EF3CFDBFF050EDB6AD1
:101A9000040EDBCF20F0050EDBCF21F031EC15F08A
:101AA0000A0E1FC0DBFF0B0E20C0DBFF0C0E21C097
:101AB000DBFF0D0E22C0DBFF040EDBCF00F0050EB6
:101AC000DBCF01F0080EDBCF02F0090EDBCF03F015
:101AD00001500318E8AE02D0033404D00250005C79
:101AE000035001582EE20A0EDBCF00F00B0EDBCFC5
:101AF00001F00C0EDBCF02F00D0EDBCF03F0246AF9
:101B0000256A200E266E410E276E00C01FF001C010
:101B100020F002C021F003C022F0F6EC15F00A0E0E
:101B20001FC0DBFF0B0E20C0DBFF0C0E21C0DBFF54
:101B30000D0E22C0DBFF040EDB2A050E01E3DB2ABB
:101B4000BBD70A0EDBCF04F00B0EDBCF05F00C0E7B
:101B5000DBCF06F00D0EDBCF07F0246A256A266A7C
:101B6000400E276E04C01FF005C020F006C021F013
:101B700007C022F0F6EC15F01FC000F020C001F005
:101B800021C002F022C003F0D950FB0FE96EFF0E16
:101B9000DA20EA6EEECF1FF0EECF20F0EECF21F08C
:101BA000EFCF22F000C024F001C025F002C026F0E3
:101BB00003C027F060EC15F022C0EDFF21C0EDFF5F
:101BC00020C0EDFF1FC0EFFFFB0EDBCF00F0FC0ECF
:101BD000DBCF01F0FD0EDBCF02F0FE0EDBCF03F01A
:101BE000246A256A200E266E410E276E00C01FF063
:101BF00001C020F002C021F003C022F078EC17F001
:101C0000010A13E0FB0EDB6AFC0EDB6A800EF36E4A
:101C1000FD0EF3CFDBFF3F0EF36EFE0EF3CFDBFFC7
:101C2000020EDB2A030E01E3DB2A020EDBCF00F0FB
:101C3000030EDBCF01F00001800E01145FE0F90E0E
:101C4000DBCFE9FFDB2AFA0EDBCFEAFF01E3DB2A79
:101C5000300EEF6EF90EDBCFE9FFDB2AFA0EDBCF99
:101C6000EAFF01E3DB2A2E0EEF6E080EDBCF00F059
:101C7000090EDBCF01F0800E011414E0020EDBCF61
:101C800002F0030EDBCF03F0080EDB50025C006EA7
:101C9000090EDB500358016E020E00C0DBFF030E7D
:101CA00001C0DBFF040EDB68050EDB68040EDBCF32
:101CB00000F0050EDBCF01F0020EDBCF02F0030EC9
:101CC000DBCF03F003500118E8AE02D0013404D09A
:101CD0000050025C0150035811E2F90EDBCFE9FF1E
:101CE000DB2AFA0EDBCFEAFF01E3DB2A300EEF6ED0
:101CF000040EDB06050E01E2DB06D8D7040EDB6A14
:101D0000050EDB6A040EDBCF00F0050EDBCF01F021
:101D1000080EDBCF02F0090EDBCF03F001500318F1
:101D2000E8AE02D0033404D00250005C03500158E6
:101D300001E3ACD0FB0EDBCF1FF0FC0EDBCF20F0BD
:101D4000FD0EDBCF21F0FE0EDBCF22F009EC17F009
:101D5000060E20C0DBFF070E21C0DBFF300EE76E52
:101D6000060EDBCF00F0070EDBCF01F0E7500026B8
:101D7000000E0122F90EDBCFE9FFDB2AFA0EDBCFE2
:101D8000EAFF01E3DB2A00C0EFFF040EDBCF00F027
:101D9000050EDBCF01F0020EDB50001803E1030E4D
:101DA000DB5001180BE1F90EDBCFE9FFDB2AFA0E5D
:101DB000DBCFEAFF01E3DB2A2E0EEF6E060EDBCF50
:101DC00020F0070EDBCF21F031EC15F00A0E1FC01A
:101DD000DBFF0B0E20C0DBFF0C0E21C0DBFF0D0E66
:101DE00022C0DBFF1FC000F020C001F021C002F0C4
:101DF00022C003F0D950FB0FE96EFF0EDA20EA6E25
:101E0000EECF1FF0EECF20F0EECF21F0EFCF22F09B
:101E100000C024F001C025F002C026F003C027F066
:101E20005FEC15F022C0EDFF21C0EDFF20C0EDFFFB
:101E30001FC0EFFF006A016A200E026E410E036EA2
:101E4000D950FB0FE96EFF0EDA20EA6EEECF1FF0DD
:101E5000EECF20F0EECF21F0EFCF22F000C024F043
:101E600001C025F002C026F003C027F049EC16F0AF
:101E700022C0EDFF21C0EDFF20C0EDFF1FC0EFFF2E
:101E8000040EDB2A050E01E3DB2A3CD7F90EDBCF7B
:101E9000E9FFFA0EDBCFEAFFEF6A0E0EE15C02E229
:101EA000E16AE552E16EE552E7CFD9FF1200D9CFE2
:101EB000E6FFE1CFD9FF060EE12602010D9DFB0EE4
:101EC000DBCF1FF0FC0EDBCF20F0FD0EDBCF21F0CF
:101ED000FE0EDBCF22F038EC17F01EC0DEFF1FC075
:101EE000DEFF20C0DEFF21C0DDFFDD52DD52FB0E34
:101EF000DBCF04F0FC0EDBCF05F0FD0EDBCF06F0F0
:101F0000FE0EDBCF07F0F90EDBCF20F0FA0EDBCFB1
:101F100021F031EC15F01FC008F020C009F021C0FD
:101F20000AF022C00BF008C024F009C025F00AC056
:101F300026F00BC027F004C01FF005C020F006C03B
:101F400021F007C022F049EC16F01FC000F020C0BD
:101F500001F021C002F022C003F0F90EDBCF14F033
:101F6000FA0EDBCF15F0166A176A15AE02D01668A6
:101F7000176814C01EF015C01FF016C020F017C05F
:101F800021F0DFCF23F0010EDBCF24F0020EDBCFF8
:101F900025F0030EDBCF26F0F2EC1BF01AC010F098
:101FA0001BC011F01CC012F01DC013F010C01EF0B9
:101FB00011C01FF012C020F013C021F046EC15F044
:101FC0001FC00CF020C00DF021C00EF022C00FF099
:101FD0000CC024F00DC025F00EC026F00FC027F075
:101FE00000C01FF001C020F002C021F003C022F0A9
:101FF0005FEC15F009EC17F0040E20C0DBFF050EB6
:1020000021C0DBFF000EE66E010EE66ED9CFE9FFC0
:10201000DACFEAFFEECFE6FFEECFE6FFEECFE6FF48
:10202000EFCFE6FFA9EC1AF0006E060EE15E00505D
:1020300002010D51800B01E0010E006E016A00509B
:10204000011012E0F80EDBCF00F0016A00BE01685B
:102050000050E66E000EE66E010EE66EE7EC08F04C
:10206000E552E552E5520CD0000EE66E010EE66E2A
:102070004FEC0AF0E552E552F3CF1CF2F4CF1DF21B
:1020800002010D51800B01E0010E006E016A00504B
:1020900001100FE0F80EDBCF00F0016A00BE01680E
:1020A0000050E66E2E0EE66E7CEC06F0E552E55230
:1020B00007D02E0EE66EE66A94EC0AF0E552E55281
:1020C000F80EDBCF00F0016A00BE01680050E66E3A
:1020D000E66A040EDBCFE6FF050EDBCFE6FFB9ECC8
:1020E0000AF0E552E552E552E552060EE15C02E2E5
:1020F000E16AE552E16EE552E7CFD9FF1200D9CF90
:10210000E6FFE1CFD9FFE652800EDF6EDF50006EB2
:10211000016A013404E200500008000E015422E27A
:10212000FE0EDBCF02F0DF500214006E016A005099
:10213000011008E0310EE66EE66A94EC0AF0E55212
:10214000E55207D0300EE66EE66A94EC0AF0E552EE
:10215000E552DF50006E016AD89001320032005023
:10216000DF6ED4D7E552E552E7CFD9FF1200D9CFC1
:10217000E6FFE1CFD9FF020EE126FE0EDB50006E36
:10218000016AF00E0016000E0116040ED8900132FE
:102190000032E804FBE1300E0024DF6EDFCF00F0F8
:1021A000016A00BE0168013404E200503908000EE3
:1021B000015408E2DFCF00F0016A00BE0168070E9B
:1021C0000024DF6EFE0EDB50006E016A0F0E00165B
:1021D000000E0116300E0026000E0122010E00C076
:1021E000DBFFDBCF00F0016A00BE0168013404E2CE
:1021F00000503908000E01540AE2070E006E010E6D
:10220000DBCFE7FF0050E726010EE7CFDBFFDFCF94
:1022100000F0016A00BE016800C0E6FF01C0E6FFF1
:1022200094EC0AF0E552E552010EDBCF00F0016AB2
:1022300000BE016800C0E6FF01C0E6FF94EC0AF0B2
:10224000E552E552680EE66EE66A94EC0AF0E55255
:10225000E552020EE15C02E2E16AE552E16EE5520E
:10226000E7CFD9FF1200D9CFE6FFE1CFD9FFFB0EB0
:10227000DBCF1FF0FC0EDBCF20F0FD0EDBCF21F01B
:10228000FE0EDBCF22F02234000E221809E6D880A1
:10229000000E1F54000E2054000E2154000E225434
:1022A0000CE2D950FB0FE96EFF0EDA20EA6EEE0663
:1022B000000EEE5AEE5AEE5ADAD7E552E7CFD9FFC2
:1022C0001200D9CFE6FFE1CFD9FF020EE126DE6A88
:1022D000DD6ADECF00F0DDCF01F0FE0EDB50000145
:1022E00001AE02D0D89003D0005C000E01580CE281
:1022F000200EE66EE66A94EC0AF0E552E552DF2A1B
:10230000010E01E3DB2AE5D7020EE15C02E2E16A9D
:10231000E552E16EE552E7CFD9FF1200D9CFE6FFD3
:10232000E1CFD9FFFE0EDB50A96EA69EA69CA6802B
:10233000F40EE66E010EE66EE66AE66A94DFE5529A
:10234000E552E552E552A85000D0E552E7CFD9FF5B
:102350001200D9CFE6FFE1CFD9FFFE0EDB50A96E08
:10236000FD0EDB50A86EA69EA684550EA76EAA0E83
:10237000A76EA682A150100B01E0010E006E016A4B
:102380000050011001E1F6D7A198A694E552E7CFDD
:10239000D9FF1200D9CFE6FFE1CFD9FFFB0EDBCF8B
:1023A000E9FFFC0EDBCFEAFFEF50006E016A005040
:1023B00001101AE0FB0EDBCFE9FFDB2AFC0EDBCFBE
:1023C000EAFF01E3DB2AEF50E66EFD0EDBCF00F003
:1023D000DB2AFE0EDBCF01F001E3DB2A0050E66EC4
:1023E000B8DFE552E552DAD7E552E7CFD9FF120060
:1023F000D9CFE6FFE1CFD9FF020EE126FD0EDBCFFC
:10240000E6FF8CDFE552DE6EDD6AD9CFE9FFDACF79
:10241000EAFFEE50ED1001E121D0DFCFE6FFE66AE2
:1024200094EC0AF0E552E552FD0EDB2AFE0E01E3C4
:10243000DB2AFD0EDBCF00F0FE0EDBCF01F0013416
:1024400004E20050FF08000E015401E207D0D9CF8A
:10245000E9FFDACFEAFFEE50ED10D0E1980EE66E1C
:102460003A0EE66EE66AE66AFEDEE552E552E552AF
:10247000E552020EE15C02E2E16AE552E16EE552EC
:10248000E7CFD9FF12008168936893809382939479
:1024900093869388938A938C938EC26A070EC16E3B
:1024A000926E896A8268800E946E9490949294944D
:1024B00094969498949A949C948E1200F50EE66EDD
:1024C00051EC1CF0E552CD92CD8E9F80D08EDB0E6C
:1024D000E66E0B0EE66E91EC1CF0E552E5529E9016
:1024E000F28CCD909D80F28EF28C1200CCDF809623
:1024F0000201046B36EC0AF002010D9F9E50200B86
:1025000001E0010E006E016A0050011005E072EC5E
:102510001CF00201176FF2D7100EE66E270EE66E62
:10252000E66AE66AA0DEE552E552E552E5520C0E97
:10253000E66EE66A94EC0AF0E552E552F00EE66EBD
:10254000490EE66E020EE66EE66A8DDEE552E55253
:10255000E552E5520201096B0A6B006B016B808644
:10256000ACEC0AF00101000E5A6F010E5B6F5AC10C
:10257000E6FF5BC1E6FF4FEC0AF0E552E552F3CF10
:102580001CF2F4CF1DF2ACEC0AF080960101000EB3
:102590005A6F010E5B6FD4C100F0D5C101F0026A21
:1025A00000C0E6FF01C0E6FF02C0E6FF5AC1E6FF39
:1025B0005BC1E6FF2AEC1CF0036E050EE15E0350E2
:1025C0005AC1E6FF5BC1E6FF4FEC0AF0E552E55267
:1025D000F3CF1CF2F4CF1DF2E80EE66E030EE66EAA
:1025E000E66AE66A40DEE552E552E552E552000E43
:1025F000E66EE66AFDDEE552E552200EE66EE66A1C
:10260000F7DEE552E552600EE66EE66AF1DEE5526F
:10261000E552800EE66EE66AEBDEE552E552ACEC82
:102620000AF0E80EE66E030EE66EE66AE66A1BDE68
:10263000E552E552E552E552808602010D8FD6EC57
:1026400004F08050080B01E0010E026E036A025094
:10265000031002E0000E01D0010E006E016A00506E
:10266000E8B08086E8A0809608EC05F0F0EC05F074
:10267000E66AE66A93EC05F0E552E552E8C100F03F
:10268000E9C101F0026A00C0E6FF01C0E6FF02C036
:10269000E6FF000EE66E010EE66E2AEC1CF0036EFD
:1026A000050EE15E0350E66A000EE66E010EE66E70
:1026B000E7EC08F0E552E552E552010EE66EE66AF7
:1026C00093EC05F0E552E552EAC100F0EBC101F0F0
:1026D000026A00C0E6FF01C0E6FF02C0E6FF000E8E
:1026E000E66E010EE66E2AEC1CF0036E050EE15E4E
:1026F0000350E66A000EE66E010EE66EE7EC08F0A7
:10270000E552E552E552020EE66EE66A93EC05F0FC
:10271000E552E552ECC100F0EDC101F0026A00C0E3
:10272000E6FF01C0E6FF02C0E6FF000EE66E010E06
:10273000E66E2AEC1CF0036E050EE15E0350E66ABD
:10274000000EE66E010EE66EE7EC08F0E552E5528B
:10275000E552040EE66EE66A93EC05F0E552E552AA
:10276000F6C100F0F7C101F0026A00C0E6FF01C047
:10277000E6FF02C0E6FF000EE66E010EE66E2AECF2
:102780001CF0036E050EE15E0350E66A000EE66E75
:10279000010EE66EE7EC08F0E552E552E552880ED0
:1027A000E66E130EE66EE66AE66A5DDDE552E55218
:1027B000E552E5528050080B01E0010E026E036AFB
:1027C0000250031002E0000E01D0010E006E016AFB
:1027D0000050E8B08086E8A080960201006B016B93
:1027E0000E6B0F6B6BDE02011A6B1B6B1E6B1F6B8C
:1027F000CD800E510F11FDE00E6B0F6B0D8F8050D1
:10280000080B01E0010E026E036A0250031002E0A1
:10281000000E01D0010E006E016A0050E8B0808603
:10282000E8A08096030EE66E280EE66E93EC05F0A7
:10283000E552E552E66AE66A1AC2E6FF1BC2E6FF07
:10284000B9EC0AF0E552E552E552E55202010D9F5E
:102850000101000E5A6F010E5B6FE2C100F0E3C18F
:1028600001F0026A00C0E6FF01C0E6FF02C0E6FF19
:102870005AC1E6FF5BC1E6FF2AEC1CF0036E050EB1
:10288000E15E03501AC200F01BC201F00A0E256E71
:10289000266A00C020F001C021F0DBEC1CF020C053
:1028A00000F021C001F0300E0026000E0122120EB1
:1028B0000101EA6A5A25E96E5B51EA2200C0EFFF86
:1028C0001AC200F01BC201F00A0E256E266A00C073
:1028D00020F001C021F0DBEC1CF01CC000F01DC09A
:1028E00001F0300E0026000E0122130E0101EA6AEB
:1028F0005A25E96E5B51EA2200C0EFFF0201186B16
:10290000196B080E185D000E19591DE2650E182589
:10291000E96E010E1921EA6EEF50E66E4B0E0101D1
:10292000016A5A25006E5B510122005002011825F0
:10293000E96E01501921EA6EE552E750EF6E182B4F
:10294000000E1923DED75AC1E6FF5BC1E6FF4FEC4C
:102950000AF0E552E552F3CF1CF2F4CF1DF204C2A7
:1029600000F0016A00BE0168005001104FE06EC126
:1029700000F0016A00BE0168450E001801E1015037
:1029800041E10201186B196B080E185D000E195910
:1029900017E26F0E1825E96E010E1921EA6EEFCFCE
:1029A00000F0016A00BE0168650E1825E96E010E8F
:1029B0001921EA6E00C0EFFF182B000E1923E4D78F
:1029C00001016D6B8150020B01E0010E006E016A86
:1029D0000050011017E1ACEC0AF0520EE66EE66A08
:1029E00094EC0AF0E552E5526F0EE66E010EE66ECB
:1029F0004FEC0AF0E552E552F3CF1CF2F4CF1DF292
:102A0000ACEC0AF00201046B01016E6B02011A2B9F
:102A1000000E1B230D8F050EE66E180EE66E93EC6E
:102A200005F0E552E552E66A650EE66E010EE66EC9
:102A3000E7EC08F0E552E552E55202010D9F010E68
:102A40001A251A6F000E1B211B6F3B0ED8801A55DA
:0E2A5000000E1B5502E21A6B1B6BCBD6120058
:022A5E00199EBF
:102A600008D0199E21AE05D0206C211EE86A2122D3
:102A7000198E21C01BF020C01AF02B6A2A6A8E0E14
:102A80001C6E1D6AF2EF17F0199E0CD0199E21AE34
:102A900009D01E6C1F1E201E211EE86A1F22202244
:102AA0002122198E21C01BF020C01AF01FC02BF06C
:102AB0001EC02AF09E0E1C6E1D6AF2EF17F0277ED4
:102AC000196A2EEC18F046EC18F019B6D6EF17F08C
:102AD00019A20AD019AA03D019BED6EF17F019A46B
:102AE000E2EF17F0DFEF17F019AA05D019ACE2EF0B
:102AF00017F0DFEF17F019A00AD019A808D019BEF7
:102B000004D019A402D0EBEF17F0EFEF17F02A6A08
:102B10001D6A2750225C296E10E31FC02BF020C0D5
:102B20001AF021C01BF022C028F024C01FF025C0DD
:102B300020F026C021F0193A09D024C02BF025C07E
:102B40001AF026C01BF027C028F0296C199E19BC6A
:102B5000198E28C01CF019B01EEF18F01A0E29604B
:102B60001EEF18F01C6A226A19A408D01F6C201EE0
:102B7000211E221EE86A20222122222219AC08D01E
:102B80002B6C1A1E1B1E1C1EE86A1A221B221C22FA
:102B90001E6A295207E02234213220321F321E32AF
:102BA000292EF9D71F502B2620501A2221501B22E4
:102BB00022501C221EC02AF0199E1CAE0BD02A6C7B
:102BC0002B1E1A1E1B1E1C1EE86A2B221A221B22F9
:102BD0001C22198E1CA006D0D8801B321A322B3230
:102BE0002A32282A28C01CF0F2EF17F0196A2EECBE
:102BF00018F046EC18F019B6D6EF17F019A205D068
:102C000019BAD6EF17F0DDEF17F019BAE9EF17F0A0
:102C100019A005D019B8D6EF17F0E9EF17F019B8D9
:102C2000DDEF17F01D6A7F0E22241C6EE86A1D225C
:102C300027501C5EE86A1D5A1A0E286E226A2A6AFC
:102C40002B6A1A6A1B6A24501F5E2550205A265090
:102C5000215A000E225A09E724501F26255020220F
:102C600026502122000E222201D02A8AD8901F3617
:102C7000203621362236D8902A362B361A361B3685
:102C8000282EE1D7215020101F10D8A42A8AF2EF55
:102C900017F0196A2EEC18F046EC18F019B6D6EFBA
:102CA00017F019A205D019B8D6EF17F0DDEF17F01D
:102CB00019AA05D019B0D6EF17F0DDEF17F019B04B
:102CC00002D019A802D0E9EF17F01D6A275022247C
:102CD0001C6EE86A1D227E0E1C5EE86A1D5A2A6A76
:102CE0002B6A1A6A1B6A26502102F4CF1BF0F3CF1D
:102CF0001AF025502102F3502B26F4501A22000E10
:102D00001B2226502002F3502B26F4501A22000ECC
:102D10001B2224502102F3502A26F4502B22000EAD
:102D20001A221B2225502002F3502A26F4502B226F
:102D3000000E1A221B2226501F02F3502A26F4509E
:102D40002B22000E1A221B2224502002F4502A2685
:102D5000000E2B221A221B2225501F02F4502A2675
:102D6000000E2B221A221B22F2EF17F0186A26AE51
:102D7000BFEF16F0256C261EE86A2622181E21AE2B
:102D8000C7EF16F0206C211EE86A2122181EDBEC2A
:102D90001CF021BED7EF16F018AE000C206C211EDF
:102DA000E86A21221C6C1D1EE86A1D22000C18BE58
:102DB000CEEF16F01988FF0C21C02BF020C02AF0AE
:102DC00020502502F4CF1FF0F3CF1EF02150260231
:102DD000F4CF21F0F3CF20F02502F3501F26F4505A
:102DE0002022E86A21222A502602F3501F26F4509E
:102DF0002022E86A212226AE02EF17F02A50205E38
:102E00002B50215A2BAE000C2550205E2650215A03
:102E1000000C196A2EEC18F019B613EF17F019A26E
:102E20000ED019B405D07F0E216EFF0E206E1FD07C
:102E3000800E216E206A1BD0216A206A18D019B03A
:102E4000FBD78F0E2260EDD77E0E2264F5D78E0E53
:102E5000225C05E0D89021322032222AF8D719A42A
:102E600006D0206C211EE86A212221AEE5D712008F
:102E7000196A2EEC18F019B642EF17F019A20FD00C
:102E800019B407D07F0E216EFF0E206E1F6E1E6ECE
:102E900025D0800E216E01D0216A000EF6D719B020
:102EA000FBD71E6A9F0E2260EBD77E0E2264F4D7FA
:102EB0009E0E225C07E0D890213220321F321E3253
:102EC000222AF6D719A40AD01E6C1F1E201E211E0E
:102ED000E86A1F222022212221AEDED7120081ECD7
:102EE00017F019B6000C19B0000C19B4000C010C45
:102EF00081EC17F019B6000C19B0000C19A4000CE5
:102F0000010C196A2EEC18F046EC18F019B61200F4
:102F100019AE08D019A004D019A802D01980120047
:102F2000199012002750225C0BE12650215C08E129
:102F30002550205C05E124501F5C02E1198012003D
:102F4000D8A002D0198E10D0225027C022F0276EB0
:102F5000215026C021F0266E205025C020F0256E7D
:102F60001F5024C01FF0246E2750225C10E0FF0F7A
:102F700009E0199019B403D019AE1984120019AEE2
:102F800019941200272AD890263225322432245050
:102F90001F5E2550205A2650215A21BEEAD7D890CC
:102FA0001F3620362136222EF8D7C8D77F0E226E44
:102FB000FF0E216E206E1F6E12007F0E19BEFF0ED7
:102FC000226E02D07F0E226E800E216E206A1F6A52
:102FD000F3D719AE04D0800E226E216AF7D7226A89
:102FE000216AF4D71B501A102B102A10F8E01DBECE
:102FF000F0D71BBE0CD01C501D10EBE0D8902A3629
:103000002B361A361B361C06D8A01D06F2D71D50CB
:10301000D4E11C28D2E02AAE11D07F0E2A1402E19E
:103020002BA00CD02B2AE86A1A221B2207E3D88097
:103030001B321A322B321C2A1C28BFE01C50C9E05C
:103040002BC01FF01AC020F01B34216E1C30226EE2
:103050002132229E19BE228EDCEF17F02136223655
:1030600002E31984197E06E11980226A216A206A26
:103070001F6A1200222803E0D88021321200D89063
:10308000213202E1198212001986120026362736F3
:1030900002E3198C197E06E11988276A266A256AD7
:1030A000246A1200272803E0D88026321200D89024
:0830B0002632EAE1198A120040
:0830B800000000000000005FB1
:1030C00000000007000700147F147F14242A7F2AC1
:1030D000122313086462364955225000050300008C
:1030E000001C2241000041221C0014083E08140864
:1030F000083E080800503000000808080808006072
:1031000060000020100804023E5149453E00427F05
:10311000400042615149462141454B311814127F0C
:103120001027454545393C4A494930017109050395
:103130003649494936064949291E003636000000FD
:1031400056360000081422410014141414140041CF
:103150002214080201510906324979413E7E1111BB
:10316000117E7F494949363E414141227F414122FA
:103170001C7F494949417F090909013E4149497A72
:103180007F0808087F00417F41002040413F017FC8
:10319000081422417F404040407F020C027F7F04A0
:1031A00008107F3E4141413E7F090909063E4151D9
:1031B000215E7F09192946464949493101017F01AC
:1031C000013F4040403F1F2040201F3F4038403FCC
:1031D00063140814630708700807615149454300E8
:1031E0007F41410002040810200041417F00040299
:1031F00001020440404040400001020400205454B9
:1032000054787F484444383844444420384444483F
:103210007F3854545418087E0901020C5252523E11
:103220007F0804047800447D40002040443D007F36
:103230001028440000417F40007C041804787C087A
:1032400004047838444444387C14141408081414D2
:10325000187C7C080404084854545420043F44401B
:10326000203C4040207C1C2040201C3C4030403C06
:1032700044281028440C5050503C4464544C4400A2
:103280000836410000007F000000413608001008A9
:1032900008100878464146782E2E2E00506F727422
:1032A00020636F6D6D203139323030206F75766557
:1032B0007274202E2E2E20537472696E6720656EF4
:1032C00020524F4D200D0A004331383A2031384604
:1032D0003235325F4E6F6B696156395F58706F726D
:1032E000745F617263686F735F3131313132302ED8
:1032F00063200D0A0045534320706F757220736F71
:10330000727469720D00200020002000200023321A
:10331000302F31312F323031312032304833304D7F
:103320003232533B41313D303131313B41323D301E
:103330003232323B41333D303333333B41343D3025
:103340003434343B41353D303535353B4C3D3031FF
:103350003031303130313B523D303030303131312D
:10336000313B20260D0A0020006563686F203A205B
:103370000A0D003138463235325F4E6F6B6961207D
:103380004C434400204E6F6B69615F4C43445F7651
:10339000392E682000203230206E6F7620203230A7
:1033A000313120202000202020202020202020201B
:1033B000202020202020002020204D504C41422061
:1033C000433138202020200020206E6F6B6961205F
:1033D000333431302E2E2E2E002E2E2E2E2E2E2E2B
:1033E0002E2E2E2E2E2E2E2E2E0020436F6D6D6132
:1033F0006E646520726563756520002020202020A2
:103400002020202020202020202020002E2E2E2EA4
:0D3410002E2E2E2E2E2E2E2E2E2E2E2E0087
:02341E00D9CF04
:10342000E6FFDACFE6FFFA0EE3CFD9FFFB0EE3CFDC
:10343000DAFFFD0EE35209E72D0EDE6EFC0EE31EF1
:10344000E32AFD0ED8B4E306E31EE652E652E65246
:10345000FD0EE124E76EFF0EE220E46EE652F70E69
:10346000E3CFE6FFF70EE3CFE6FF7FEC1AF0F90EAD
:10347000E124E96EFF0EE220EA6E6FEC1AF00AE139
:103480006CEC1AF009E16FEC1AF008E16CEC1AF040
:1034900007E108D07AEC1AF075EC1AF07AEC1AF021
:1034A00075EC1AF07AEC1AF0DE6AF90EE126FF0EDE
:1034B000E222FF0EE3CFDAFFE552FF0EE3CFD9FFA2
:1034C000E552FC0EE124E96EFF0EE220EA6EEECF3B
:1034D000F3FFEFCFF4FF1200EF380F0B1200EF50A5
:1034E0000F0B02E1EE52D8841200EF380F0B300FB1
:1034F000DE6E1200EE500F0B300FDE6E1200FC0E6F
:10350000E3CFE9FFFD0EE3CFEAFF100EE66EEE6AB1
:10351000EE6AEF6AD890FD0EE336FE0EE336ED3626
:10352000ED36EF36FF0EE30609E0A0EC1AF0EE529E
:10353000A0EC1AF0EE52A0EC1AF0EDD7E56E1200F6
:10354000030EEF24E8B6EF6E300EEF24E8BEEF6E08
:10355000000CD9CFE6FFDACFE6FFF80EE3CFD9FFB4
:10356000F90EE3CFDAFFE652E652E652E652E652B1
:10357000FB0EE124E76EFF0EE220E46EE652F30E4E
:10358000E3CFE6FFF30EE3CFE6FFF30EE3CFE6FF74
:10359000F30EE3CFE6FF2EEC1BF0F50EE124E96E0F
:1035A000FF0EE220EA6E1BEC1BF019E11EEC1BF093
:1035B00018E11BEC1BF017E11EEC1BF016E11BECF5
:1035C0001BF015E11EEC1BF014E11BEC1BF013E1EA
:1035D0001EEC1BF012E11BEC1BF011E112D024ECED
:1035E0001BF029EC1BF024EC1BF029EC1BF024EC65
:1035F0001BF029EC1BF024EC1BF029EC1BF024EC55
:103600001BF029EC1BF0DE6AF50EE126FF0EE2222C
:10361000FF0EE3CFDAFFE552FF0EE3CFD9FFE5520D
:10362000FA0EE124E96EFF0EE220EA6EEECFF3FF20
:10363000EFCFF4FF1200EF380F0B1200EF500F0B1B
:1036400002E1EE52D8841200EF380F0B300FDE6E1D
:103650001200EE500F0B300FDE6E1200FA0EE3CFA9
:10366000E9FFFB0EE3CFEAFF200EE66EEE6AEE6A9C
:10367000EE6AEE6AEF6AD890FB0EE336FC0EE33694
:10368000FD0EE336FE0EE336ED36ED36ED36ED3665
:10369000EF36FF0EE3060FE05DEC1BF0EE525DEC43
:1036A0001BF0EE525DEC1BF0EE525DEC1BF0EE52A7
:1036B0005DEC1BF0E1D7E56E1200030EEF24E8B6D7
:0C36C000EF6E300EEF24E8BEEF6E000C41
:0436CC000E0EF66E7A
:1036D000000EF76E000EF86E02010900F550A56F9E
:1036E0000900F550A66F03E1A56701D03DD00900A0
:1036F000F550A06F0900F550A16F0900F550A26FB9
:1037000009000900F550E96E0900F550EA6E09005C
:1037100009000900F550A36F0900F550A46F0900D6
:103720000900F6CFA7F2F7CFA8F2F8CFA9F2A0C20E
:10373000F6FFA1C2F7FFA2C2F8FF0201A35302E104
:10374000A45307E00900F550EE6EA307F8E2A407C2
:10375000F9D7A7C2F6FFA8C2F7FFA9C2F8FF020176
:0A376000A507000EA65BBFD71200FC
:06376A00D9CFE6FFDACF23
:10377000E6FFE1CFD9FFE2CFDAFFAC6AAB6AFD0E1C
:10378000DBB0AC88DBA202D0AC8CAB8CDBB4AC8EF3
:10379000DBA602D0AB8801D0AB8ADBA802D0AC8418
:1037A00001D0AC949E98DBAC02D09D8A01D09D9A4A
:1037B0009E9ADBAE02D09D8801D09D98FB0EDB5017
:1037C000AF6EAC8AAB8E949C948EAC50100B04E020
:1037D000AC50800B01E1948CE552E5CFDAFFE7CFE6
:0437E000D9FF1200FB
:0C37E4001E502302F3CF1AF0F4CF1BF0AC
:1037F0002402F3501B26000EF4201C6E1E502502DE
:10380000F3501C26000EF4201D6E1E502602F350AD
:103810001D261F502302F3501B26F4501C22000EBD
:103820001D221F502402F3501C26F4501D221F504D
:103830002502F3501D2620502302F3501C26F4507D
:103840001D2220502402F3501D2621502302F35044
:043850001D2612001F
:0C385400FB0EE3CFF6FFFC0EE3CFF7FF06
:10386000FD0EE3CFF8FFFE0EE3CFE9FFFF0EE3CF3F
:10387000EAFFE9CFF3FFEACFF4FF0900F5CFEFFF4E
:10388000EE66FBD71200FE0EE3CFE9FFFF0EE3CF9B
:10389000EAFFF36AF46AEE5203E0F34AF42AFBD734
:0238A000120014
:0E38A200D9CFE6FFDACFE6FFE1CFD9FFE2CFC4
:1038B000DAFFFD0EDB507E0BCD6EFD0EDBAC02D0D1
:1038C000CD8E01D0CD9ECF6ACE6A9E90DBAE02D067
:1038D0009D8001D09D90CD80E552E5CFDAFFE7CF06
:0438E000D9FF1200FA
:0C38E400D9CFE6FFDACFE6FFE1CFD9FF35
:1038F000E2CFDAFFE652F20E0101FC17ABAC03D0C7
:10390000FC91ABB0FC81ABB4FC85ABB2FC87AE5094
:10391000DF6EDF50E552E552E5CFDAFFE7CFD9FFA2
:02392000120093
:0E392200D9CFE6FFDACFE6FFE1CFD9FFE2CF43
:10393000DAFFE652E652FC0EDBCFDEFFDBCFDDFF27
:10394000010EDB50CF6EDF50CE6EE552E552E552F0
:0A395000E5CFDAFFE7CFD9FF120040
:06395A00FF0EE350336E86
:10396000EF0E01D0F30EE76EE72EB4EF1CF00C0E55
:10397000326EE76AE72EBAEF1CF0322EB9EF1CF078
:08398000332EB2EF1CF012001F
:08398800D9CFE6FFDACFE6FF1C
:10399000E1CFD9FFE2CFDAFFACAC04D0AC900101AB
:1039A000FCB3AC80FD0EDB50AD6EE552E5CFDAFF27
:0639B000E7CFD9FF120071
:0A39B6001D6A1C6A100EE76ED8901F
:1039C000203621361C361D3625501C5C26501D58CD
:1039D00005E325501C5E26501D5A202AE72EF0D7FD
:0239E0001200D3
:0E39E200000EF36E00EE00F0060E01D812008B
:1039F000EA6002D0EE6AFCD7F350E9601200EE6A8A
:023A0000FCD7F1
:0E3A020015EE00F025EE00F0F86A199C66EC57
:0E3A10001BF003EC00F076EC12F0FBD7120076
:023A1E00F36A49
:103A2000F46AF32A0F0B05E0D890F336F436E80475
:043A3000FBE11200A4
:0C3A34003138463235325F4E6F6B6961ED
:103A400056395F58706F72745F617263686F735F2D
:103A500031313F3F3F3F2E632020737472696E67A0
:103A600020656E2052414D0D000000000000000056
:103A70000000000000000000000000000000000046
:103A80000000000000000000000000000000000135
:103A90003132333435363738003132333435363716
:103AA000380030303030303030300000000000005E
:103AB0000000000000000000000000000000000006
:103AC00000000000000000000000000000000000F6
:103AD00000000000000000000000000000000000E6
:103AE00000000000000000000000000000000000D6
:103AF00000000000000000000000000000000000C6
:103B000000000000000098329C32C832F5320633C3
:103B100008330A330C330E3367336933733384331A
:103B20009533A633B733C833D933EA33FB330C3478
:020000040030CA
:01000100FA04
:01000200F409
:01000300FEFE
:01000600FBFE
:0200000400F00A
:1000000050726F6A65743A203138463235325F6E0D
:100010006F6B69612E6D63702020202020200D0001
:10002000506F727420436F6D20313932303062204E
:100030002620496E697420484152442E20200D002C
:100040002E2E2E2E2E2E2E2E2E2E2E2E2E2E2E2ED0
:1000500020203C4553433E206578697420200D00E4
:1000600041766563205541525420484152445741DE
:1000700052452E2E2E2E2E2E2E2E2E2E2E200D00C2
:10008000313846323532206176656320626F6F7495
:100090006C6F6164657220313932303062200D003E
:1000A0007061756C666A756A6F40667265652E660A
:1000B00072202020202020202020202020200D0021
:1000C0004D504C4142204944452056382E3633206D
:1000D000204331382076332E33372E3031200D0037
:1000E0004E6F6B69612033343130203936783438C3
:1000F00020384C783136636172730D0A00000000BD
:00000001FF
